:1000000053C06DC06CC06BC06AC069C068C067C0B7
:1000100066C0CCC764C063C062C061C060C05FC05E
:100020005EC05DC05CC040C13FC13EC13DC13CC17E
:1000300008C23AC1E2C1DCC24CC327C226C249C3CE
:1000400024C223C246C345C344C304C317C300002C
:100050000000370034003100000000003800350097
:1000600032000000000036003300300004040404B5
:100070000404040402020202020203030303030352
:10008000010204081020408001020408102001022F
:100090000408102000000000000000000003040518
:1000A000000000000000000011241FBECFE5D4E0D6
:1000B000DEBFCDBF10E0A0E6B0E0E8E2F3E102C0B1
:1000C00005900D92A036B107D9F710E0A0E6B0E098
:1000D00001C01D92A03BB107E1F764D723C990CFBF
:1000E0000F931F93880F991F672B59F08C010659A6
:1000F0001F4FF801808160E040D8F801808161E005
:100100000AC08C0106591F4FF801808161E035D883
:10011000F801808160E011D81F910F9108950F932D
:100120001F93182F062F60E028D861E070E080E070
:1001300090E0ACD781E062E041E02FE18ED861E051
:1001400070E080E090E0A2D781E062E041E0202F03
:1001500084D861E070E080E090E098D7812F61E082
:100160000CD81F910F9108950F931F93CF93DF9396
:10017000EC018B018091680090916900892B09F452
:1001800067C0C830D10554F4C430D1058CF4209731
:1001900089F1C130D10509F09CC241C0CE30D105F2
:1001A00039F0C331D10541F02B9709F092C20EC04E
:1001B000CE01B80195DF8DC280919200909193009D
:1001C000892B09F086C283E090E00DC061157105AE
:1001D00061F081E090E0909393008093920083E03F
:1001E00090E062ED70E09BDF74C210929300109279
:1001F00092006FC26115710551F080E090E06CE8EB
:1002000070E08DDF109291001092900062C2809198
:10021000900090919100892B09F05BC214C0611588
:10022000710551F080E090E062ED70E078DFD093EE
:100230009100C09390004DC28091900090919100E8
:10024000019709F046C280E090E060E070E0CBCF1B
:1002500080918A0090918B00892BF1F020918C0085
:1002600030918D00C9018F779070892BA9F4C90155
:10027000019790938D0080938C00E199FECF9FBBF6
:100280008EBB8FEF8DBB0FB6F894E29AE19A0FBE4A
:1002900010928B0010928A00FE01C431D10508F043
:1002A00018C2ED5EFF4F099480918A0090918B00F7
:1002B000892B09F450C020918C0030918D002130A1
:1002C000310509F406C260918E0070918F006115AE
:1002D000710551F4E199FECF3FBB2EBB1DBA0FB69D
:1002E000F894E29AE19A0FBE012BC1F0E199FECF9A
:1002F0003FBB2EBBE09A4DB3E199FECF3FBB2EBB77
:1003000081E090E002C0880F991FCA95E2F7482B60
:100310004DBB0FB6F894E29AE19A0FBECB0101965D
:1003200090938F0080938E00069709F0D2C11092AF
:100330008F0010928E00E199FECF3FBB2EBBE09A5A
:100340008DB3882309F4C5C12F5F3F4F30938D00D3
:1003500020938C00BEC1209751F480919800909119
:100360009900019721F40115110521F5B2C1C130A1
:10037000D10551F480919A0090919B00019721F44E
:1003800001151105F9F4A5C1C230D10531F48091F0
:10039000940090919500019749F0C330D10551F434
:1003A0008091960090919700019761F401151105D5
:1003B00091F48FC1C430D10529F480919E009091B1
:1003C0009F0007C0C630D10531F480919C00909108
:1003D0009D00892B19F4CE01B80182DE012B09F4AE
:1003E00078C180918C0090918D00019709F071C1C6
:1003F00010928D0010928C006CC1012BE9F080915D
:100400009C0090919D000B972CF086E090E061E0BD
:1004100070E004C086E090E060E070E061DE809112
:100420009C0090919D00019664E170E054D79093F8
:100430009D0080939C004DC110929D0010929C00E5
:1004400048C1012BE9F080919E0090919F000B978D
:100450002CF084E090E061E070E004C084E090E083
:1004600060E070E03DDE80919E0090919F000196DB
:1004700064E170E030D790939F0080939E0029C183
:1004800010929F0010929E0024C1012B09F421C1FB
:10049000CA30D10519F482E090E010C0CB30D1050C
:1004A00019F481E890E00AC0CD30D10519F481E05B
:1004B00091E004C02E9731F481E891E090938D0093
:1004C00080938C0080918A0090918B00892B09F495
:1004D00080C0FFC0E199FECF3FBB2EBBE09A6DB359
:1004E00070E06170707080E090E03EDE20918C00E2
:1004F00030918D00E199FECF3FBB2EBBE09A6DB3EA
:1005000070E0759567956170707081E090E02CDE09
:1005100020918C0030918D00E199FECF3FBB2EBB26
:10052000E09A6DB370E07595679575956795617004
:10053000707082E090E018DE20918C0030918D0088
:10054000E199FECF3FBB2EBBE09A6DB370E053E064
:10055000759567955A95E1F76170707083E090E04A
:1005600003DE20918C0030918D00E199FECF3FBBDE
:100570002EBBE09A6DB370E044E0759567954A959F
:10058000E1F76170707084E090E0EEDD20918C0006
:1005900030918D00E199FECF3FBB2EBBE09A6DB349
:1005A00070E036E0759567953A95E1F76170707087
:1005B00086E090E0D9DD80918C0090918D000196CD
:1005C00090938D0080938C0064E170E080E090E077
:1005D0005DD580918C0090918D00E199FECF9C01BA
:1005E0009FBB8EBBE09A8DB38F3F09F073CF71C074
:1005F000012B09F46EC080918A0090918B002091AC
:100600008C0030918D00892BB1F02130310509F437
:1006100060C0E199FECF3FBB2EBB8FEF8DBB0FB605
:10062000F894E29AE19A0FBE10928B0010928A0021
:1006300081E090E00AC02130310509F44AC081E030
:1006400090E090938B0080938A0090938D0080932C
:100650008C003FC010929500109294001092970069
:1006600010929600003511051CF482E090E013C052
:100670000B3A110574F183E090E01FC010929900CD
:100680001092980010929B0010929A00003511056C
:100690007CF480E090E061E070E022DD083211053A
:1006A000C4F481E090E0909395008093940011C091
:1006B0000B3A110574F081E090E061E070E010DD2C
:1006C000033D110534F081E090E090939700809312
:1006D0009600DF91CF911F910F910895DF92EF92D5
:1006E000FF920F931F93CF93DF93D82EF62EE42E15
:1006F00010E001E0C0E0D0E0602F6E218D2D3DD5EF
:10070000000F8F2D60E039D58091A0009091A1005D
:10071000E7D4169584E068D59695982F8827979505
:100720008795180F8F2D61E028D52196C830D10507
:1007300019F78091A0009091A100D2D4812FDF9170
:10074000CF911F910F91FF90EF90DF900895FF924E
:100750000F931F93CF93DF9386E060E00ED585E083
:1007600090E067E070E041E0B9DF85E090E067E0AD
:1007700070E042E4B3DFF82E83E5F81659F083E722
:10078000F81659F081E4F81671F41092670010928F
:10079000660009C081E090E002C082E090E09093A2
:1007A00067008093660085E090E067E070E040E0DD
:1007B00095DF8091660090916700181619064CF03D
:1007C0008091680090916900892B19F402E010E093
:1007D00002C006E010E0C0E0D0E085E090E067E015
:1007E00070E040E07BDFFE01E05AFF4F80832196FE
:1007F000C017D10794F386E061E0BFD48F2D90E05D
:10080000DF91CF911F910F91FF9008950F931F9348
:10081000CF93DF939CDF83E061E0AFD480E061E0C1
:10082000ACD46091600070E001E010E060277127B7
:100830006170707089E090E097DC6091600070E01A
:100840007695679560277127617070708FE090E0F2
:100850008BDC6091600070E0769567957695679582
:1008600060277127617070708CE090E07DDC609192
:10087000600070E033E0769567953A95E1F7602780
:1008800071276170707088E090E06EDC60916000AC
:1008900070E024E0769567952A95E1F76027712747
:1008A0006170707080E090E05FDC6091600070E0EB
:1008B00095E0769567959A95E1F7602771276170C5
:1008C000707083E090E050DC6091600070E086E042
:1008D000769567958A95E1F760277127617070704A
:1008E00081E090E041DC60E070E08091600087FD95
:1008F00002C061E070E082E090E036DCC09166000A
:10090000D0916700C130D10509F06BC060916100E2
:1009100070E06C277D27617070708BE090E024DCC4
:100920006091610070E0769567956C277D27617016
:1009300070708AE090E018DC6091610070E076955C
:100940006795769567956C277D276170707086E056
:1009500090E00ADC6091610070E0A3E07695679515
:10096000AA95E1F76C277D276170707087E090E0B1
:10097000FBDB6091610070E0F4E076956795FA9595
:10098000E1F76C277D27617070708DE090E0ECDB03
:100990006091610070E0E5E076956795EA95E1F792
:1009A0006C277D276170707085E090E0DDDB6091E1
:1009B000610070E056E0769567955A95E1F76C27EF
:1009C0007D276170707084E090E0CEDB60E070E0C5
:1009D0008091610087FD02C061E070E08EE090E0F0
:1009E0006CC06091610070E001E010E06027712749
:1009F000617070708BE090E0B7DB6091610070E037
:100A00007695679560277127617070708EE090E031
:100A1000ABDB6091610070E07695679576956795A0
:100A200060277127617070708AE090E09DDB6091B3
:100A3000610070E023E0769567952A95E1F76027DD
:100A40007127617070708DE090E08EDB60916100C5
:100A500070E094E0769567959A95E1F760277127A5
:100A60006170707087E090E07FDB6091610070E002
:100A700085E0769567958A95E1F760277127617023
:100A8000707085E090E070DB6091610070E0B6E02E
:100A900076956795BA95E1F7602771276170707058
:100AA00084E090E061DB60E070E08091610087FDB0
:100AB00002C061E070E086E090E056DB8091660065
:100AC000909167001816190634F080916800909193
:100AD0006900892BC1F06091620080E190E070E0D4
:100AE00043DB6091630081E190E070E03DDB609169
:100AF000640082E190E070E037DB6091650083E1A3
:100B000090E070E031DBDF91CF911F910F9108955C
:100B100086E060E032D385E090E067E070E041E09D
:100B2000DDDD85E090E067E070E043E4D7DD85E05F
:100B300090E067E070E040E0D1DD85E090E067E0C4
:100B400070E041E0CBDD85E090E067E070E040E000
:100B5000C5DD86E061E011D364E670E080E090E0FE
:100B600095D286E060E009D385E090E067E070E030
:100B700041E0B4DD85E090E067E070E044E4AEDDA4
:100B800085E090E067E070E040E0A8DD85E090E07F
:100B900067E070E041E0A2DD85E090E067E070E0B2
:100BA00040E09CDD85E090E067E070E040E096DDAD
:100BB00085E090E067E070E040E090DD85E090E067
:100BC00067E070E040E08ADD85E090E067E070E09B
:100BD00040E084DD86E061E0D0D264E670E080E051
:100BE00090E054D286E060E0C8D285E090E067E013
:100BF00070E041E073DD85E090E067E070E043E4A1
:100C00006DDD85E090E067E070E040E067DD85E065
:100C100090E067E070E040E061DD85E090E067E053
:100C200070E040E05BDD85E090E067E070E040E090
:100C300055DD85E090E067E070E040E04FDD85E065
:100C400090E067E070E040E049DD85E090E067E03B
:100C500070E040E043DD86E061E08FD20895CF93FD
:100C6000DF931092950010929400109297001092CA
:100C70009600109299001092980010929B0010928A
:100C80009A00109293001092920010929D00109280
:100C90009C0010929F0010929E001092A300109250
:100CA000A20060ED77E080E090E0F0D184E060E0C9
:100CB00044D285E061E041D286E061E03ED287E047
:100CC00061E03BD288E060E038D289E060E035D274
:100CD0008AE060E032D28BE060E02FD28CE060E00E
:100CE0002CD28DE060E029D283E160E026D283E05F
:100CF00061E023D280E061E020D282E061E01DD299
:100D000081E061E01AD289E061E037D28AE061E0F7
:100D100034D28BE061E031D28CE061E02ED28DE004
:100D200061E02BD286E061E028D287E061E025D245
:100D300085E061E022D280E590E09093A10080936D
:100D4000A0001092690010926800C0E0D0E0FFDCC3
:100D5000409168005091690020E030E0809160008F
:100D600087FD02C021E030E0C901840F951F9093F8
:100D70006900809368002196C436D10541F78B3510
:100D800091055CF081E090E09093690080936800A9
:100D9000EAE6F0E08FEF9FEF0BC084E190E09093E4
:100DA000A1008093A0001092690010926800F0CF1B
:100DB0008193919320E0EA38F207D1F7809168009F
:100DC00090916900892B01F189E090E09093870070
:100DD000809386008AE090E0909375008093740081
:100DE0008BE090E090937900809378008CE090E025
:100DF00090937300809372008DE090E09093770061
:100E00008093760085DE67C089E090E090936B0068
:100E100080936A008AE090E090936D0080936C006C
:100E20008BE090E090936F0080936E008CE090E0F8
:100E300090937100809370008DE090E09093730028
:100E40008093720083E190E0909377008093760026
:100E500083E060E092D161E070E080E090E016D144
:100E600081E062E041E02FE1F8D161E070E080E0F4
:100E700090E00CD181E062E041E02FEFEED161E043
:100E800070E080E090E002D183E061E076D168EC30
:100E900070E080E090E0FAD080E060E06ED161E048
:100EA00070E080E090E0F2D081E062E041E02FE18C
:100EB000D4D161E070E080E090E0E8D081E062E0D1
:100EC00041E02FEFCAD161E070E080E090E0DED039
:100ED00080E061E052D110928B0010928A00109253
:100EE0008F0010928E00E199FECF8FE790E09FBBBC
:100EF0008EBBE09A8DB38F3F69F0E199FECF8FE70B
:100F000090E09FBB8EBB8FEF8DBB0FB6F894E29A3B
:100F1000E19A0FBEE199FECF8FEF90E09FBB8EBBB1
:100F2000E09A8DB38F3F69F0E199FECF8FEF90E0AB
:100F30009FBB8EBB8FEF8DBB0FB6F894E29AE19A00
:100F40000FBEE199FECF8FE791E09FBB8EBBE09A89
:100F50008DB38F3F69F0E199FECF8FE791E09FBBA2
:100F60008EBB8FEF8DBB0FB6F894E29AE19A0FBE5D
:100F7000E199FECF8FEF91E09FBB8EBBE09A8DB3DE
:100F80008F3F69F0E199FECF8FEF91E09FBB8EBB61
:100F90008FEF8DBB0FB6F894E29AE19A0FBEDF9106
:100FA000CF910895ABD05BDE31DCFECF1F920F9264
:100FB0000FB60F9211242F938F939F93AF93BF93EC
:100FC0008091A4009091A500A091A600B091A700E7
:100FD0000196A11DB11D8093A4009093A500A0933C
:100FE000A600B093A7008091A8009091A900A091BD
:100FF000AA00B091AB008050904CAF4FBF4F809390
:10100000A8009093A900A093AA00B093AB0027C0BA
:101010008091A8009091A900A091AA00B091AB0086
:1010200080589E43A040B0408093A8009093A900B0
:10103000A093AA00B093AB008091AC009091AD005A
:10104000A091AE00B091AF000196A11DB11D80939B
:10105000AC009093AD00A093AE00B093AF00809130
:10106000A8009091A900A091AA00B091AB0081586E
:101070009E43A040B04060F6BF91AF919F918F9189
:101080002F910F900FBE0F901F901895EF92FF9227
:101090000F931F937B018C018FB7F8944091AC00A4
:1010A0005091AD006091AE007091AF008FBF2FB72F
:1010B000F8948091AC009091AD00A091AE00B091F9
:1010C000AF002FBF841B950BA60BB70BE816F906D4
:1010D0000A071B0760F71F910F91FF90EF9008958B
:1010E000019759F0FC01EE0FFF1FEE0FFF1F329723
:1010F0008FB7F8943197F1F78FBF0895789483B73D
:10110000826083BF83B7816083BF89B7816089BFF5
:101110008EB582608EBD8EB581608EBD8FB58160CB
:101120008FBD85B5846085BD85B5806485BD329AE7
:10113000319A309A379A1AB80895282F30E0C901A9
:1011400080589F4FFC01949124593F4FF90184919D
:10115000882391F0E82FF0E0EE0FFF1FE25BFF4FD6
:10116000A591B491662329F48C91909589238C9351
:1011700008958C91892B8C930895482F50E0CA01D3
:101180008C569F4FFC012491CA0180589F4FFC014F
:10119000949144595F4FFA013491332321F1222372
:1011A00081F0233019F48FB58F7704C0243021F4F7
:1011B0008FB58F7D8FBD05C0253019F485B58F7D26
:1011C00085BDE32FF0E0EE0FFF1FE85AFF4FA5911A
:1011D000B491662329F48C91909589238C9308957A
:1011E0008C91892B8C930895682F70E0CB018C56DD
:1011F0009F4FFC012491CB0180589F4FFC014491EB
:1012000064597F4FFB019491992319F420E030E059
:1012100022C0222381F0233019F48FB58F7704C0C8
:10122000243021F48FB58F7D8FBD05C0253019F492
:1012300085B58F7D85BD892F90E0880F991F8E59C8
:101240009F4FFC01A591B4918C9120E030E0842364
:1012500011F021E030E0C9010895BF92CF92DF92F2
:10126000EF92FF920F931F93CF93DF93E82EF62E0A
:10127000B42EC0E0D0E0022F10E087E0C82ED12CC1
:10128000BB2041F4B8010C2E02C0759567950A94F5
:10129000E2F70AC0B6016C1B7D0BC80102C0959530
:1012A00087956A95E2F7BC0161708E2D66DF8F2D00
:1012B00061E063DF8F2D60E060DF2196C830D105EB
:1012C000F9F6DF91CF911F910F91FF90EF90DF9092
:1012D000CF90BF90089597FB092E07260AD077FD7F
:1012E00004D00CD006D000201AF4709561957F4F81
:1012F0000895F6F7909581959F4F0895AA1BBB1B03
:1013000051E107C0AA1FBB1FA617B70710F0A61B05
:10131000B70B881F991F5A95A9F780959095BC0126
:08132000CD010895F894FFCF00
:00000001FF
